:102338002020202020202020202020200D0A002AD4
:102348004D3A2053656C6674657374206F6B0D0A83
:10235800002A573A2053656C667465737420666169
:10236800696C65640D0A002A52454144590D0A00FA
:1023780000022F002F2A00AB20015E1601D21102A5
:102388005A0C02780B02960A02B60902D70802F91B
:1023980007031C06033F05036404038B0303B2020F
:0623A80003DA0104040049
:10145B00906F157401F0906F15E0FD64126024ED30
:10146B0075F003A42478F582E43423F583E493FA2E
:10147B00740193FBC3EF9BEE9A4008906F15E00449
:10148B00F080D3ED75F003A42478F582E43423F5D2
:10149B0083C37401939FFFE4939EFEE4FCFD7BE802
:1014AB007A03F9F81204EDC8ECC8C9EDC9CAEECA43
:1014BB00CBEFCB906F15E0FF75F003A4247AF58288
:1014CB00E43423F583E493FDEF75F003A42477F55F
:1014DB0082E43423F583E493C39DFFE49400FEE49C
:1014EB00FCFD1204EDECC0E0EDC0E0EEC0E0EFC09F
:1014FB00E0906F15E0FF75F003A42475F582E434DA
:10150B0023F583E493FC740193FDEF75F003A4249E
:10151B0078F582E43423F583C37401939DFFE49340
:10152B009CFEE4FCFDF8F9CAEECACBEFCBD0E0FF92
:10153B00D0E0FED0E0FDD0E0FC120578EEC0E0EF8D
:10154B00C0E0906F15E075F003A4247AF582E434C3
:10155B0023F583E493FFE4FCFDFE7BE87A03F9F8C3
:0C156B001204EDD0E02FFFD0E03EFE2285
:1022BF00201175906F74E05407906F0CF0C3940366
:1022CF004066E064076061D2117F011230D6E4905E
:1022DF006F0CF07F017D127B031231C5301706E5BD
:1022EF006860F980397F017D0E7B031231C530178D
:1022FF0006E56860F980277F017D0A7B021231C5F0
:10230F00301706E56860F98015906F0CE004F0E077
:10231F00B403C07F0112319A7F0A1230D6227F0296
:09232F0012319A7F0A1230D62205
:10131B003012030213F5E56864036009E568640B9A
:10132B00600302145AD378D5E6954F18E6954E40D4
:10133B000A906F13E4F0A304F0803BAF4FAE4E1254
:10134B00145BEEC0E0EFC0E078D4E6FE08E6FF12D7
:10135B00145BCCEECCCDEFCDD0E0FFD0E0FEC3EDF7
:10136B009FFFEC9EFE906F13F0A3EFF04E70079073
:10137B006F13F0A304F0D201E4906F0CF0906F1395
:10138B00E0FAA3E0FB7C007D0AFFCEEACE12043626
:10139B00906F0CE0240DF582E4346FF583EDF07C57
:1013AB00007D0ACFEBCFCEEACE120436906F13EE50
:1013BB00F0A3EFF0906F0CE004F0E0B405BF906F7A
:1013CB000C7404F0906F0CE0FFF46015740D2FF5A6
:1013DB0082E4346FF583E07008906F0CE014F080BA
:1013EB00E3EF04906F12F0D212227F1E1230D67FE1
:1013FB00017D327B041231C53017043016FA227F7F
:10140B000A1230D6906F12E014906F0CF0906F0CA4
:10141B00E0240DF582E4346FF583E0700B7F017DE2
:10142B000B7B041231C58016906F0CE0240DF582F6
:10143B00E4346FF583E0FF7D0B7B011231C5301770
:10144B00043016FA22906F0CE0FF14F0EF70BE22FE
:10213E00D2AF122FFA12310812000E12302D1231B8
:10214E00F91231741200031221C512305D7BFF7A31
:10215E002379381200C912316A122C4650107BFFB7
:10216E007A2379471200C97F0112319A800B7BFFC7
:10217E007A2379591200C9D211122021906EE7E00C
:10218E00FF122BD4122B9B1228EC906EE8E0FEA3CC
:10219E00E0FF122A5B7BFF7A23796F1200C9C2120D
:1021AE00C211301603122F8B12131B906EDFE060DC
:0721BE00F11222BF80EC22A8
:03000B000223AE1F
:1023AE00C0E0C0F0C083C082C0D075D008C28CAF70
:1023BE008CEFFEAD8AED255F78D7F6E55E3E18F61A
:1023CE00F58C08E6F58AD28CD56309906EDEE0F5C1
:1023DE00631227CFD5621B906EDEE0F5620561E5D4
:1023EE006170020560E56145607007E56860037520
:1023FE006805E5686404600F1218951226A8121E6F
:10240E0026122A9E121F84D0D0D082D083D0F0D034
:02241E00E032AA
:102A5B00E4FCFDFB7AC079A8F81204ED7BE07A2E3A
:102A6B0079007800122A17C374129FF55FE49EF564
:102A7B005E906EDEE0F563F562E4F560F561E58985
:102A8B0054F04401F589758CFF758AFFC2B9D2A940
:032A9B00D28C22B8
:0C312400906EDEE0F562E4F560F56122DB
:1028EC00E5C520E3FB75C50775C50FE5C530E4FBF1
:1028FC00AFC6EF75F004A4FFAEF0E5C5C4131354D6
:10290C00037C002FF53CEC3EF53BE4F53AE53A252B
:10291C00E024C0F8A63B08A63CE53C2527F527E5B6
:10292C003B3526F526053AE53AB40AE1E4F53922B9
:10189500C0D075D008E5C520E3FBE4F5C575C508DE
:1018A500F543754401E5436408700302196AE5C50B
:1018B50030E4FB85C62885C53DE5436407600EE534
:1018C500C520E3FBE54304F5C54408F5C5E52875E2
:1018D500F004A4FFAEF0E53DC4131354037C002FC0
:1018E500F546EC3EF545E54325E02429F8A64508EF
:1018F500A646906EDDE055446060AF28122C7FAFA0
:101905003D122C7FE543B406088545418546428056
:1019150049E54364077043E53925E024C1F8C3E58B
:101925002796F527E5261896F526E53925E024C0FE
:10193500F8A64508A646E5462527F527E5453526B3
:10194500F526FEAF277C007D0A1204368E248F25EE
:101955000539E539B40A03E4F5390543E54425E0DD
:10196500F5440218AA300F1EE4A2C492E4A2C5925F
:10197500E5A29692E6A29792E72568C4F53EAF3EAA
:0D198500122C7F853E40C294D294D0D02217
:10249100C0D075D008300F65906EE7E0FD7C0090EC
:1024A1006EF2E0FB24FFFFE434FFFE120422EF246E
:1024B10001FFE43EFEC3E51F9FF51FE51E9EF51ECD
:1024C1008B3FE53F6021E51EF583E51FF582E0C402
:1024D10054F02568C4F0906EE7E0251FF51FE43540
:1024E1001EF51E153F80DB906EE7E024FFFFE4340C
:1024F100FFFEC3E51F9FF51FE51E9EF51ED0D022EE
:0D311700E4F576F577F578C219122C0D223B
:1026A800C0D075D008E56860572019541230C3406F
:1026B8004F906EE7E02404906F05F0906F05E0609E
:1026C8003F20133C122D208F7512002E0577E577D9
:1026D800700205767004E5766480701CF576F577EF
:1026E8000578E578B40C04D21980151230B0E57875
:1026F80020E005122C0D8008906F05E014F080BBD7
:03270800D0D0220C
:102B9B00E4906FB2F0906EF2E075F00584906FB137
:102BAB00F0E4906FB3F0906FAD1206500000000090
:102BBB0074FF78D4F608F6E4906FB4F0F569906F73
:092BCB00ABF0F568A374FFF022E1
:102FE000C0D075D008756801AF68122DAEC29012BE
:0A2FF00031177F0212319AD0D0226F
:0B315400C291906EDEE0906FABF022A5
:0B315F00C292906EDEE0906FABF02299
:1011B000C0D075D008E4906F05F020C604E044016B
:1011C000F020C707906F05E04402F0906FACE0FF9D
:1011D000906F05E0FE6F603BEE7025906FBAE0FF08
:1011E00060051231A2802C906FB9E0FF64036004A7
:1011F000EFB404051231A2801A7F0112319A8013D4
:10120000906F05E030E0077F011231A280057F0278
:101210001231A2906F05E0906FACF0300B1EA294DB
:10122000300C01B34016C21A123124906EDBE0FE7E
:10123000A3E0FF122D54122FE00213182010030216
:101240001318906EDAE0C4F8540FC868FF906ED996
:10125000E0C454F048FEC3E54D9FFDE54C9EFCE51F
:1012600042C4F8540FC868FFE541C454F048FED3A7
:10127000EF9DEE9C4037906FB2E070030213189020
:101280006FB1E014F0E06003021318D21A906FAD52
:1012900012065000000000E4906FB2F0906EF2E091
:1012A00075F00584906FB1F0123124806B906FB1AE
:1012B000E004F0C21A906FADE0F8A3E0F9A3E0FA01
:1012C000A3E0FBE8C0E0E542C4F8540FC868FFE5BE
:1012D00041C454F048FEC3EF954DFFEE954CFE33EC
:1012E00095E0FDFCD0E0F8EB2FFFEA3EFEE93DFD86
:1012F000E83CFC906FAD120644906EF2E0FF906FF8
:10130000B2E004F06F7011906EE2E0FEA3E0FF1215
:0B1310002D54122FE0122491D0D022A7
:101EDF00C0D075D008906FADE0F8A3E0F9A3E0FA99
:101EEF00A3E0FBE8C0E0E542C4F8540FC868FFE583
:101EFF0041C454F048FEC3EF954DFFEE954CFE33B1
:101F0F0095E0FDFCD0E0F8EB2FFFEA3EFEE93DFD4A
:101F1F00E83CFC906FAD120644300E387F007E0017
:101F2F007D007C00906FADE0F8A3E0F9A3E0FAA389
:101F3F00E0FBD312060A401C906ED8E0FFD3E56198
:101F4F009FE5609400400D123154756802AF68121E
:101F5F002DAE801E300D1B906EEEE0FEA3E065618E
:101F6F007003E5606E700B12315475680AAF68121A
:051F7F002DAED0D022C0
:10242000C0D075D008906FABE0600614F07002D297
:1024300091300E3C906EE5E0FEA3E0FFC3E54F9FB8
:10244000FFE54E9EFEC3E5259FE5249E5007E490E0
:102450006FB3F0801B906F03E0FF906FB3E004F068
:102460006F700D12315F756803AF68122DAE801E5C
:10247000300D1B906EF0E0FEA3E065617003E56037
:102480006E700B12315F75680BAF68122DAED0D035
:012490002229
:0F30F900906FABE0600814F07004D291D2922275
:101E2600C0D075D008E5687003021EB4E4F5647589
:101E36006701E56464086065E56425E024F3F582DE
:101E4600E4346EF583E0FEA3E08E65F566F4700378
:101E5600E565F4603EE56955677015E56165667090
:101E660004E56065657009E5674269AF6412298813
:101E7600E5695567601DE5662401FFE43565FEEFFB
:101E860065617003EE6560700AE567F45269AF64D8
:101E96001229D00564E56725E0F5678095C3E52539
:101EA60078D596E52418965005A62408A625E56853
:101EB60014601614601814601A24F9601114601363
:101EC600240B70121211B0800D121EDF800812242E
:091ED6002080031230F9D0D02263
:102BD400CBEFCBEBFD7C007E3A7F98120436CDEB35
:102BE400CD7C001204228E1A8F1B74002FF582EE06
:102BF4003434AF82F5188F197E347F008E1C8F1DFC
:092C04008E1E8F1FD213C2142290
:102C7F00201933C213051FE51FAC1E7002051E1469
:102C8F00F5828C83EFF0E51F65197004E51E65185A
:102C9F007006751E34751F00E51F651D7004E51E57
:072CAF00651C7002D2142223
:102D2000C214051DE51DAE1C7002051C14F5828E33
:102D300083E0FFE51D65197004E51C6518700675D4
:102D40001C34751D00E51F651D7004E51E651C70B3
:042D500002D2132276
:102D5400C3E51F9FF51DE51E9EF51CC3E51D9400EC
:102D6400E51C9434400BD3E51D9519E51C951840DA
:0E2D74000CE51B251DF51DE51A351CF51C226E
:101C79002573202562752025627520257520257517
:101C8900202575202575202563202562752025636B
:101C99002025632025630D0A00632069676E2025CE
:101CA9007520257520257520257520257520257514
:101CB9002025752025750D0A006320786D6974202B
:101CC900257520256275202562750D0A006320633C
:101CD90068616E202562750D0A00632067707320A4
:101CE9002562750D0A00696E646578006572617315
:101CF90065006F6666006F6E002A56455253494F5C
:101D09004E3A20522D4441532056332E360D0A00A7
:101D190063210063207264617300632069676E0048
:101D29006320786D69740063206368616E006320C5
:101D390067707300633F006300632000677073205E
:101D4900007265736574002A453A20756E6B6E6F73
:091D5900776E20636D640D0A0031
:08000300E4F57EC216C21522CD
:100AF600906F0CEBF0A3EAF0A3E9F0300B13300C87
:100B060008906F297401F0800D906F297402F080AF
:100B160005E4906F29F0906F0CE0FBA3E0FAA3E0E8
:100B2600F91203BA643F6003020BDC906F0FE0F921
:100B3600A3E0FAA3E0906F34C9F0A3EAF0A3E9F0CA
:100B4600906EDEE0906F37F0906EDDE0906F38F0DB
:100B5600906ED9E0FFA3E0906F39CFF0A3EFF0904D
:100B66006EE5E0FFA3E0906F3BCFF0A3EFF0906E51
:100B7600EEE0FFA3E0906F3DCFF0A3EFF0906EF0B4
:100B8600E0FFA3E0906F3FCFF0A3EFF0300F047FBC
:100B96003180027F30906F41EFF0906F29E0906FC7
:100BA60042F03010047F3180027F30906F43EFF0C7
:100BB600300E047F3180027F30906F44EFF0300DAD
:100BC600047F3180027F30906F45EFF07BFF7A1C07
:100BD60079791200C922906F0CE0FBA3E0FAA3E03A
:100BE600F91203BAFF123073500C906F0DE475F0D2
:100BF600011204C180E0E4906F28F0906F0CE0FBD6
:100C0600A3E0FAA3E0F9121685906F28E025E02408
:100C160012F582E4346FF583EEF0A3EFF0906F0CDB
:100C2600E0FBA3E475F0011204D7A9F0FA1203BAA7
:100C3600FF12307350E7906F28E004F0E0B40BBB6E
:100C4600906F13E0906EDEF0906F15E0906EDDF021
:100C5600906F16E0FFA3E0906ED9CFF0A3EFF0906F
:100C66006F18E0FFA3E0906EE5CFF0A3EFF0906F72
:100C76001AE0FFA3E0906EEECFF0A3EFF0906F1CAA
:100C8600E0FFA3E0906EF0CFF0A3EFF0906F1EE0D0
:100C9600FEA3E0FFEE4F24FF920FA3E0FEA3E0FFCA
:100CA600EE4F24FF920BEF64014E7003D38001C315
:100CB600920C906F22E0FEA3E0FFEE4F24FF92100D
:100CC600A3E0FEA3E0FFEE4F24FF920EA3E0FEA3F7
:090CD600E0FFEE4F24FF920D2215
:10179300906F0CEBF0A3EAF0A3E9F01203BA643FF5
:1017A300600302182A7BFF7A1C79A2906EF3E0FF94
:1017B300A3E0906F34CFF0A3EFF0906EF5E0FFA3BA
:1017C300E0906F36CFF0A3EFF0906EF7E0FFA3E069
:1017D300906F38CFF0A3EFF0906EF9E0FFA3E090A5
:1017E3006F3ACFF0A3EFF0906EFBE0FFA3E0906FB2
:1017F3003CCFF0A3EFF0906EFDE0FFA3E0906F3ECF
:10180300CFF0A3EFF0906EFFE0FFA3E0906F40CF27
:10181300F0A3EFF0906F01E0FFA3E0906F42CFF0F1
:10182300A3EFF01200C922906F0CE0FBA3E0FAA330
:10183300E0F91203BAFF123073500C906F0DE47588
:10184300F0011204C180E0E4906F0FF0906F0CE0A0
:10185300FBA3E0FAA3E0F9121685906F0FE025E0F1
:1018630024F3F582E4346EF583EEF0A3EFF0906F8A
:101873000CE0FBA3E475F0011204D7A9F0FA1203FC
:10188300BAFF12307350E7906F0FE004F0E0B40832
:02189300BB2276
:101D6200906F0CEBF0A3EAF0A3E9F01203BAB43FD0
:101D7200297BFF7A1C79C2906EE0E0FFA3E0906FAE
:101D820034CFF0A3EFF0906EEAE0906F36F0906FF0
:101D920004E0906F37F01200C922906F0CE0FBA3B1
:101DA200E0FAA3E0F91203BAFF123073500C906FFD
:101DB2000DE475F0011204C180E0E4906F15F0901B
:101DC2006F0CE0FBA3E0FAA3E0F9121685906F1501
:101DD200E025E0240FF582E4346FF583EEF0A3EF03
:101DE200F0906F0CE0FBA3E475F0011204D7A9F0A8
:101DF200FA1203BAFF12307350E7906F15E004F045
:101E0200E0B403BB906F0FE0FFA3E0906EE0CFF071
:101E1200A3EFF0906F12E0906EEAF0906F14E090F2
:041E22006F04F02237
:10270B00906F0CEBF0A3EAF0A3E9F0906F0CE0FBF9
:10271B00A3E0FAA3E0F91203BAB43F127BFF7A1CD1
:10272B0079D6906EEDE0906F34F01200C922906F65
:10273B000CE0FBA3E0FAA3E0F91203BAFF1230732B
:10274B00500C906F0DE475F0011204C180E0906F96
:10275B000CE0FBA3E0FAA3E0F9121685906EEDEF07
:02276B00F0225A
:10276D00906F0CEBF0A3EAF0A3E9F0906F0CE0FB97
:10277D00A3E0FAA3E0F91203BAB43F127BFF7A1C6F
:10278D0079E3906EDFE0906F34F01200C922906F04
:10279D000CE0FBA3E0FAA3E0F91203BAFF123073C9
:1027AD00500C906F0DE475F0011204C180E0906F34
:1027BD000CE0FBA3E0FAA3E0F9121685906EDFEFB3
:0227CD00F022F8
:1006F9007B017A6E799A7D20122FA9906F0FEBF00A
:10070900A3EAF0A3E9F04A70047F0180027F009018
:100719006F1CEFF0605F7B017A6E7999121685C8BC
:10072900ECC8C9EDC9CAEECACBEFCB906EEBE0FEBF
:10073900A3E0FFE4FCFD1204EDC8ECC8C9EDC9CA89
:10074900EECACBEFCB906EDBE0FEA3E0FFE4FCFD4D
:10075900EB2FFFEA3EFEED39FDEC38FC906F1212EB
:100769000644906EEBE0FEA3E0FFE4FCFD906F16FB
:1007790012064480767B017A6E7999121685C8EC47
:10078900C8C9EDC9CAEECACBEFCB906EE7E0FFE46A
:10079900FCFDFE1204EDC8ECC8C9EDC9CAEECACB0E
:1007A900EFCB906EDBE0FEA3E0FFE4FCFDEB2FFF57
:1007B900EA3EFEED39FDEC38FC906F1212064490CA
:1007C9006F0FE0FBA3E0FAA3E0F9121685C8ECC8A5
:1007D900C9EDC9CAEECACBEFCB906EE7E0FFE4FCE6
:1007E900FDFE1204ED906F16120644906F12E0FCA4
:1007F900A3E0FDA3E0FEA3E0FF780F1206318F7896
:10080900906F12E0FCA3E0FDA3E0FEA3E0FFEE542D
:100819007FFEE48E768F771230B0906F1CE060090E
:10082900E4906F1AF0A3F0800B120026906F1AEE75
:10083900F0A3EFF0E4906F0CF0A3F0906F0CE0FEE2
:10084900A3E0FFE4FCFD906F16E0F8A3E0F9A3E054
:10085900FAA3E0FBC3120620606C123130906F0ED0
:10086900EFF0906F1CE06014906F0EE0FF906F1B2B
:10087900E02FF0906F1AE03400F08018906F1AE0C2
:10088900FEA3E0FF906F0EE0FD122243906F1AEE77
:10089900F0A3EFF0906F0EE0FF1231920577E57744
:1008A900700205767004E57664807009F576F5774F
:1008B90005781230B0906F0DE004F07006906F0C5F
:1008C900E004F0020844906F1CE07013906F1AE086
:1008D900FEA3E0FF1231B8906F1AEEF0A3EFF0908B
:1008E9006F1AE0FF123192906F1BE0FF12319222D2
:10308800D3EF648094B95007EF24D0FEFF8004EF9B
:0430980024A9FF2246
:10199200906F0CEBF0A3EAF0A3E9F0906F1374FFE1
:1019A200F0A3741CF0A374EFF0A3E4F0A37405F0A9
:1019B200122641EF7003122891906F1374FFF0A367
:1019C200741CF0A374F5F0A3E4F0A37405F0906F17
:1019D2000CE0FBA3E0FAA3E0F9122641EF70041237
:1019E2002D8222906F1374FFF0A3741CF0A374FB7A
:1019F200F0A3E4F0A37403F0906F0CE0FBA3E0FA11
:101A0200A3E0F9122641EF7003C21522906F1374FE
:101A1200FFF0A3741CF0A374FFF0A3E4F0A374021C
:101A2200F0906F0CE0FBA3E0FAA3E0F9122641EF7D
:101A32007003D21522906F0CE0FBA3E0FAA3E0F949
:101A42001203BAFF122E565043906F0CE0FBA3E034
:101A5200FAA3E0F99000011203D3FF123088CDEF10
:101A6200CD906F0CE0FBA3E0FAA3E0F91203BAFFFA
:101A7200123088EFC454F02DFF906F0FF0122E7FBA
:0D1A8200906F0DE475F0021204C180A922DE
:0431E900122EE92297
:0A316A007BFF7A1D79021200C922D2
:1008F900906F1374FFF0A3741DF0A37419F0A3E4AF
:10090900F0A37402F07B017A6E7998122641EF7098
:1009190004120CDF22906F1374FFF0A3741DF0A36F
:10092900741CF0A3E4F0A37406F07B017A6E799845
:10093900122641EF7018906F0F74FFF0A3741DF029
:10094900A3741CF07B017A6E799E120AF622906FCD
:100959001374FFF0A3741DF0A37423F0A3E4F0A3B0
:100969007405F07B017A6E7998122641EF700A7B43
:10097900017A6E799D12179322906F1374FFF0A379
:10098900741DF0A37429F0A3E4F0A37406F07B01AD
:100999007A6E7998122641EF700A7B017A6E799EF8
:1009A900121D6222906F1374FFF0A3741DF0A374DB
:1009B90030F0A3E4F0A37406F07B017A6E79981203
:1009C9002641EF700A7B017A6E799E12270B2290DD
:1009D9006F1374FFF0A3741DF0A37437F0A3E4F050
:1009E900A37405F07B017A6E7998122641EF700A9B
:1009F9007B017A6E799D12276D22906F1374FFF037
:100A0900A3741DF0A3743DF0A3E4F0A37402F07B7A
:100A1900017A6E7998122641EF7018906F0F74FF62
:100A2900F0A3741DF0A37440F07B017A6E799912DA
:100A39000AF622906F1374FFF0A3741DF0A3744299
:100A4900F0A3E4F0A37402F07B017A6E7998122680
:100A590041EF7018906F0F74FFF0A3741DF0A37429
:100A690040F07B017A6E7999120AF622906E98E02D
:100A7900B464041206F922906F1374FFF0A3741D75
:100A8900F0A37445F0A3E4F0A37404F07B017A6E3B
:100A99007998122641EF700A7B017A6E799C1219B6
:100AA9009222906F1374FFF0A3741DF0A3744AF09F
:100AB900A3E4F0A37405F07B017A6E7998122641BC
:100AC900EF70041231E922906E98E0B46904121AA9
:100AD9008F22906E98E0B4760412316A22906E9853
:0D0AE900E060097BFF7A1D79501200C922E0
:102F8B0010160280107568047F0112319A7F1E1291
:0E2F9B0030D61208F93015E81220B580E32276
:102CB600C0D0EF20E72CEF640A6027EF640D6011A7
:102CC6007498257EF582E4346EF583EFF0057E80F8
:102CD600117498257EF582E4346EF583E4F0D216FD
:052CE600F57ED0D022B4
:102501002A4D4553534147453A2053746F72696EC2
:102511006720706172616D657465727320696E20E8
:10252100464C4153480D0A002A4D455353414745F6
:102531003A2046696E69736865642073746F7269C5
:102541006E670D0A00000001C001C802000C001BEB
:1025510001000019003C03FFFFFFFFFFFFFFFFFF2A
:0D256100FFFFFFFFFFFFFF00000A01000069
:0A317400757C25757D461210292296
:10102900902546E49324FF920BA3E49324FF920CAA
:10103900A3E49324FF9210A3E493906EDDF090252E
:101049004AE49324FF920FE4906EE7F07F80EF600B
:1010590014906EDDE05F6007906EE7E02402F0EF28
:10106900C313FF80E9300F06906EE7E004F0902586
:101079004BE493906EDEF090254CE493906EE4F08F
:1010890090254DE493FF740193906ED9CFF0A3EFAF
:10109900F090254FE493FF740193906EE5CFF0A390
:1010A900EFF0906EDEE0FBFD7C007E037FE812042A
:1010B90036906EE8EEF0A3EFF0906EE7E0FA8BF071
:1010C900A4FF906EEBE5F0F0A3EFF0EB1313543FA0
:1010D900906EF2F0FB906F03F0902551E49324FF9A
:1010E900920EA3E49324FF920DA3E493FF7401935A
:1010F900906EEECFF0A3EFF0902555E493FF7401C5
:1011090093906EF0CFF0A3EFF0902557E493906E93
:10111900D8F0906EE4E0FF7E00906EEBE0FCA3E077
:10112900FD120422906EDBEEF0A3EFF0EBFF7E00E0
:10113900EAFD7C00120422E02F906EE3F0906EDB52
:10114900E03E906EE2F0E4FFEF25E02458F582E4FA
:101159003425F583E493FC740193FDEF25E024F332
:10116900F582E4346EF583ECF0A3EDF00FEFB408EB
:10117900D7902568E493FF740193906EE0CFF0A3B4
:10118900EFF090256AE493906EEAF090256BE49372
:10119900906F04F090256CE493906EEDF090256DBE
:0711A900E493906EDFF022D9
:100CDF00A20BE433857D82857C83F0A20CE433A3E1
:100CEF00F0A210E433857D82857C83A3A3F0906E00
:100CFF00DDE0857D82857C83A3A3A3F0A20FE4337F
:100D0F00FFE57D2404F582E4357CF583EFF0906EEA
:100D1F00DEE0FFE57D2405F582E4357CF583EFF019
:100D2F00906EE4E0FFE57D2406F582E4357CF583E3
:100D3F00EFF0906ED9E0FEA3E0FFE57D2407F5828A
:100D4F00E4357CF583EEF0A3EFF0906EE5E0FEA3C3
:100D5F00E0FFE57D2409F582E4357CF583EEF0A311
:100D6F00EFF0A20EE433FFE57D240BF582E4357C32
:100D7F00F583EFF0A20DE433FFE57D240CF582E45B
:100D8F00357CF583EFF0906EEEE0FEA3E0FFE57D9E
:100D9F00240DF582E4357CF583EEF0A3EFF0906E31
:100DAF00F0E0FEA3E0FFE57D240FF582E4357CF54E
:100DBF0083EEF0A3EFF0906ED8E0FFE57D2411F500
:100DCF0082E4357CF583EFF0E4906F0CF0906F0CBC
:100DDF00E0FF6408603BEF25E024F3F582E4346E16
:100DEF00F583E0FEA3E0FFE57D2412F582E4357C78
:100DFF00F583C083C082906F0CE0D082D08375F0F2
:100E0F0002120681EEF0A3EFF0906F0CE004F08079
:100E1F00BC906EE0E0FEA3E0FFE57D2422F582E4C6
:100E2F00357CF583EEF0A3EFF0906EEAE0FFE57D01
:100E3F002424F582E4357CF583EFF0906F04E0FF16
:100E4F00E57D2425F582E4357CF583EFF0906EED9A
:100E5F00E0FFE57D2426F582E4357CF583EFF09005
:100E6F006EDFE0FFE57D2427F582E4357CF583EF27
:100E7F00F07BFF7A2579011200C9122CEB7BFF7AE8
:070E8F002579291200C92298
:10202100E5C520E3FB75C50675C50EE5C530E4FBC6
:10203100AFC6EF75F004A4FFAEF0E5C5C4131354A9
:10204100037C002FF54DEC3EF54CE5C520E3FB7517
:10205100C50775C50FE5C530E4FBAFC6EF75F004E4
:10206100A4FFAEF0E5C5C4131354037C002FF54A59
:10207100EC3EF549F54E854A4FD21AE4F547F5484D
:10208100FFEF25E0247BF582E4346FF583E54CF026
:10209100A3E54DF0E54D2548F548E54C3547F547B5
:1020A1000FEFB410DCE4F54BE5482401F54DE435C0
:0420B10047F54C2281
:1027CF00301A5EE5482401F54DE43547F54CE54BED
:1027DF0025E0247BF582E4346FF583E0FEA3E0FF70
:1027EF00C3E5489FF548E5479EF547E54B25E024AF
:1027FF007BF582E4346FF583E541F0A3E542F0E524
:10280F00422548F548E5413547F547054BE54BB4BB
:10281F001003E4F54B85494E854A4F85244985259C
:02282F004A223B
:102FFA00D21B43878075985AE589540F4420F58976
:0A300A00758DFFD28ED2BCD2AC222D
:03002300022E04A6
:102E0400C0E0C0F0C083C082C0D075D01030980735
:102E1400AF99C298122CB6309904C299D21BD0D063
:092E2400D082D083D0F0D0E0325E
:08319200301BFDC21B8F9922C6
:0731AA00CEEFCE123192229C
:102E2D00E5C520E3FB8FC5EF4408F5C5E5C530E4E6
:102E3D00FBAFC6EF75F004A4FFAEF0E5C5C41313E8
:092E4D005403FDE5F0EF4DFF22F6
:102EE900E4F5A8F5E8F5B8F5F875780FE578A2E006
:102EF90092B5A2E192B3A2E292B4A2E392B202FF26
:022F0900FE22A6
:1030B000E578A2E092B5A2E192B3A2E292B4A2E3D3
:0330C00092B222A7
:0C313000E5764480857782F583E0FF227D
:10002E0090D3557499F090ACAA7466F090D3557431
:10003E0090F0E575F5F0E576D2E7F583E577F58294
:0D004E00E5F0F0E0A2E730F701B340F72243
:102C0D00E578A2E092B5A2E192B3A2E292B4A2E37A
:102C1D0092B290D3557499F090ACAA7466F090D39B
:102C2D00557480F090D3557499F090ACAA7466F0F9
:092C3D009080007414F0D21C22F6
:1030C300301C0D908000E020E703D38001C3921CE5
:0330D300A21C221A
:102CEB0075780C122C0D1230C340FB75780D123019
:102CFB00B0E4F576F577857782857683E0F5751206
:102D0B00002E0577E57770020576E5777004E5769A
:052D1B00648070E2225B
:0331F900C21C22D3
:03005B0002256E0D
:10256E00C0E0C0D0C2CC742D25C9F5C9301758159E
:10257E0050E5507052E55670128552FCC2C0F551AE
:10258E00755601E55425E0F550803CE55664017022
:10259E002375FCFFD2C00551E5516553700E3018FE
:1025AE0007F556855550801FC217801B755602754C
:1025BE0050028013E556B4020E8552FCC2C0755609
:0C25CE0001E55425E0F550D0D0D0E032FB
:10302D0075FCFFD2C075FE0B75528075EA0DC2FCA2
:08303D00D2EC75550AC21722FE
:102EA300C217A202921875FCFFD2C08F53E4F556E5
:102EB300CEEDCE8EFECEEBCE8E54855550EF600216
:032EC300D2172201
:0631BF00D202122EA32231
:0631C500C202122EA3223B
:08319A007D0B7B011231BF2205
:0831A2007D327B041231BF22D3
:1030D600C21775FCFFD2C08F55E4F556855550D200
:0230E6001722AF
:10157700413A2534752025347520253475202534C6
:10158700752025347520253475202534752025349C
:101597007520443A25303262782043433A25632543
:1015A700632042573A25630D0A002A4D3A20615FAE
:1015B7007374203D2025750D0A002A4D3A206128B5
:1015C7003029203D2025750D0A002A573A20615FF2
:1015D70073743D25752C2061303D25752028672DB6
:1015E70073772064697361626C6564290D0A002A48
:1015F7004D3A2070283029203D2025750D0A002AF4
:10160700573A20502072616E6765205B25752C253F
:10161700755D0D0A002A573A204257206572726F8E
:1016270072202842572064697361626C6564290DD2
:101637000A002A573A206E6F2069676E2025626478
:101647000D0A002A573A206E6F20786D69740D0ACB
:10165700002A573A206E6F206770730D0A002A57C9
:101667003A2064726F677565206572720D0A002AE9
:0E167700573A206D61696E206572720D0A008F
:0731B100EF60031F80FA220A
:101A8F001016028003021B86E4A2C492E0A2C59244
:101A9F00E1A29692E2A29792E3F57BE4FF122E2D3C
:101AAF00EFC0E0EEC0E07F01122E2DEFC0E0EEC0E0
:101ABF00E07F02122E2DEFC0E0EEC0E07F03122E6A
:101ACF002DEFC0E0EEC0E07F04122E2DEFC0E0EE50
:101ADF00C0E07F05122E2DEFC0E0EEC0E07F0612B2
:101AEF002E2DEFC0E0EEC0E07F07122E2D906F423B
:101AFF00EEF0A3EFF0906F40D0E0F0A3D0E0F090C5
:101B0F006F3ED0E0F0A3D0E0F0906F3CD0E0F0A3B8
:101B1F00D0E0F0906F3AD0E0F0A3D0E0F0906F38C3
:101B2F00D0E0F0A3D0E0F0906F36D0E0F0A3D0E09B
:101B3F00F0906F34D0E0F0A3D0E0F07BFF7A15790E
:101B4F0077906F44E57BF030C6047F6380027F6F30
:101B5F00906F45EFF030C7047F6380027F6F906F07
:101B6F0046EFF03094047F6F80027F63906F47EFF2
:081B7F00F01200C9021A8F22C6
:102F6C00A2029293E4F579F57A7F781231B1057A61
:0F2F7C00E57A70020579E57A640A457970EB22EF
:100E9600E4906F11F0906F0CF0A3F0906F10F0D209
:100EA60002122F6C7F06122E2D906F0DE02FF09000
:100EB6006F0CE03EF0C202122F6C906F10E004F04F
:100EC600E0B420DB906F0CE0FEA3E0FF7C007D2009
:100ED60012048B906F0CEEF0A3EFF07BFF7A15797E
:100EE600B1906F34EEF0A3EFF01200C9E4906F0EEC
:100EF600F0A3F0A3F07F06122E2D906F0FE02FF0D7
:100F0600906F0EE03EF0906F10E004F0E0B420E544
:100F1600906F0EE0FEA3E0FF7C007D2012048B9014
:100F26006F0EEEF0A3EFF07BFF7A1579C1906F3468
:100F3600EEF0A3EFF01200C9906F0EE0FEA3E0FF03
:100F4600906F0CE0FCA3E0FDC39FFFEC9EFEC3EF99
:100F5600942DEE64809480502D7BFF7A1579D19084
:100F66006F34ECF0A3EDF0906F0EE0FFA3E0906F0E
:100F760036CFF0A3EFF01200C97F061231A2C210DD
:100F8600906F117406F0E4906F0CF0A3F0906F1060
:100F9600F07F07122E2D906F0DE02FF0906F0CE072
:100FA6003EF0906F10E004F0E0B420E5906F0CE0A6
:100FB600FEA3E0FF7C007D2012048B906F0CEEF008
:100FC600A3EFF07BFF7A1579F6906F34EEF0A3EF7E
:100FD600F01200C9906F0CE0FEA3E0FFC3947DEE13
:100FE60064809482400BD3EF94DBEE64809483405C
:100FF6002C7BFF7A167906906F34EEF0A3EFF0A300
:101006007402F0A3747DF0A37403F0A374DBF012F2
:1010160000C97F051231A2906F117405F0906F110F
:03102600E0FF22C6
:101B8700E4906F0CF0300B1EA294300C01B340169A
:101B97007BFF7A16791C1200C97F031231A2C20B90
:101BA700906F0C7403F0E4906F0DF0906F0DE0FFF1
:101BB7006408606AEF25E024F3F582E4346EF58368
:101BC700E0FCA3E0F47002ECF4604B12313C401FE0
:101BD7007F041231A27BFF7A167939906F0DE004EA
:101BE700906F34F01200C9906F0C7404F080279046
:101BF7006F0DE0FF12293C401D7F041231A27BFFCD
:101C07007A167939906F0DE004906F34F01200C99D
:101C1700906F0C7404F0906F0DE004F0808D906E5F
:101C2700E0E07002A3E060201231CB401B7F04127A
:101C370031A27BFF7A16794A1200C9E4906EE0F070
:101C4700A3F0906F0C7404F0906EDFE0601E12300A
:101C57001440197F041231A27BFF7A1679581200BB
:101C6700C9E4906EDFF0906F0C7404F0906F0CE095
:021C7700FF224A
:102C4600D201121B87906FB9EFF06002C201120E1B
:102C560096906FBAEFF06002C20120C60B7BFF7A36
:102C66001679651200C9C20120C70B7BFF7A167957
:092C7600761200C9C201A201227C
:10000E00E4FF74B52FF582E4346FF58374FFF00FBF
:05001E00EFB404EE2226
:0C313C00EFC31325E02441FF122FC52231
:10293C00906F0EEFF0E0FFC31325E02441FF7B0105
:10294C007A6F7910906F177401F0122AE1906F0F63
:10295C00EFF0906F0EE054012402FF74017E00C86A
:10296C00EFC8088005C333CE33CED8F9FF906F1073
:0C297C00E0FDE4EF5D6003D38001C322A6
:10298800CEEFCEEEC313FF24B5F582E4346FF583A2
:10299800C083C082E0FDEE5401FC7401C8ECC80895
:1029A8008002C333D8FCF45DD082D083F0EF25E0F9
:1029B8002440FFEEC31324B5F582E4346FAD82FCE6
:0829C8007B01D202122B6022F8
:1029D000CEEFCEEEC313FF24B5F582E4346FF5835A
:1029E000C083C082E0FDEE5401FC7401C8ECC8084D
:1029F0008002C333D8FC4DD082D083F0EF25E02491
:102A000040FFEEC31324B5F582E4346FAD82FC7B46
:072A100001D202122B60222B
:10305D00E4F57FFF746E2FF582E4346FF583E4F0B1
:06306D000FEFB40DEF228D
:10301400906F0E7450F07F587C6F7D0E7B01D2024E
:09302400122B607F50122FC5220F
:102E7F00906F10EFF0A37450F07F587C6F7D117B33
:102E8F0001D202122B607F507C6F7D107B01D2022A
:042E9F00122B602270
:1020B500906F0E7453F07F587C6F7D0E7B01D202BA
:1020C500122B607F537B017A6F790D906F17740126
:1020D500F0122AE1906F0CEFF0A3E0D394104003C7
:1020E5007410F0906F0DE0604FA37451F07F587C31
:1020F5006F7D0E7B01D202122B607F517B017A6FBF
:10210500799B906F0DE0906F17F0122AE1906F0C9C
:10211500EFF0E4F0906F0DE0FF906F0CE0FE6F6064
:1021250017749B2EF582E4346FF583E0FF1231922C
:09213500906F0CE004F080DC2244
:10289100E4906F10F0906F127457F07F587C6F7D49
:1028A100127B01D202122B607F577B017A6F799BD9
:1028B100906F177410F0122AE1906F11EFF0E4F0AD
:1028C100906F11E0FF64106017749B2FF582E43460
:1028D1006FF583E0FF1231AA906F11E004F080E000
:0B28E100906F10E004F0E0B408AB22A0
:102D8200906F127456F07F587C6F7D127B01D202D5
:102D9200122B60906F107442F07F567C6F7D107B17
:0C2DA20001D202122B60906F11EFF022A2
:102DAE00906F06EFF0906F087454F07F587C6F7D33
:102DBE00087B01D202122B607F547C6F7D067B0153
:0B2DCE00C202122B60906F07EFF02292
:102A9E00C0D075D008906EDFE06035057F906EDE99
:102AAE00E0657F702BF57F906F067455F07F587C34
:102ABE006F7D067B01D202122B607F557B017A6FF0
:102ACE007968906F17740DF0122AE1906F05EFF090
:032ADE00D0D02233
:1021C500D21DE4F557F558F559906EDEE0FF75F030
:1021D5000A84755C00F55DEFC313755A00F55B90D5
:1021E5006EE0E0FEA3E0FF4E6053906F597404F07B
:1021F500E4A3F0FCFDF8F9CAEECACBEFCBFF7EC035
:102205007DA8122A177B107A0079007800122A1708
:10221500EF14906F5BF0906F04E075F080A4FF9071
:102225006EEAE02F906F5CF0906EEDE0906F5DF0E0
:0E2235007F607C6F7D597B05D202122B6022E8
:0631CB007F60122FC522F7
:1025DA00C0E0A3E558F0A3E559F0A3E52AF0A3E586
:1025EA002CF0A3E52EF0A3E530F0A3E532F0A3E545
:1025FA0034F0A3E536F0A3E538F0A375F000E52939
:10260A0042F0E52B232342F0E52DC442F0E52FC426
:10261A00232345F0F0A375F000E53142F0E53323BA
:10262A002342F0E535C442F0E537C4232345F0F0F0
:07263A00A3E540F0D0E0220F
:101F8400C0D075D008906EE0E07002A3E070030248
:101F9400201E301D09E5686005E4F557C21DE557AC
:101FA400FB7A00AC5CAD5DFFCEEACE120436ED4C9C
:101FB400705C906EDFE0601DAC5AAD5BCFEBCFCEB2
:101FC400EACE120436ED4C700C906F05741CF0A32D
:101FD4007402F0800A906F05740FF0A37401F090FE
:101FE4006F05E0906F59F0906F06E0906F5AF01211
:101FF40025DA7F607C6F7D59906F05E0FBC2021289
:102004002B60E56860080559E559700205580557C5
:0D201400906EDEE065577002F557D0D022C7
:102F2C000000CC01D8011400F0013C002800E401A1
:102F3C00A0016C007800B40150009C018801440091
:050026007EFF7FFF22B8
:10224300CBEFCBCAEECAC9EDC9E9540FFFEAEB6F76
:10225300540F25E0FFE433FE742C2FF582EE342F68
:10226300F583EAC4F854F0C868FEEBC4540F48FF82
:10227300EE540FFEE4936EFA7401936FFBCFE9CF34
:10228300EFC4540F540FFFEAEF6B540F25E0FFE444
:1022930033FE742C2FF582EE342FF583EAC4F85401
:1022A300F0C868FEEBC4540F48FFEE540FFEE493EE
:0C22B3006EFA7401936FFBCEEACEFF229E
:0731B800EEF4FEEFF4FF222C
:10283100FF31EDFF317EFF3188FF2F0BFF31D1FFDB
:102841002EC6FF31D7FF31F1FF3045FF31DDFF2FBC
:102851004CFF309CFF31F5FF31FCFF31FDFF31FEB4
:10286100FF31FFFF3200FF3201FF3202FF3203FF6F
:102871003204FF3205FF3206FF3207FF3208FF3113
:10288100E3FF31E3FF31E3FF31E3FF31E3FF31E305
:0F310800D296D29775D8C575DBECD2BDD2AD2269
:102FC500E4F56F8F6DD21ED2DDFF122DD9EF641897
:0B2FD5006004EFB44003D38001C3226E
:102B6000906F13ECF0A3EDF08C838D827880EBFEF8
:102B70006006E0F6A308DEFA8B6F8F6DD21ED2DD01
:102B800030020DCFEBCF122DD9906F15EFF08005ED
:0B2B9000E4906F15F0906F15E0FF223D
:102AE100906F14EBF0A3EAF0A3E9F0CEEFCEA3E0F0
:102AF100FFF56F8E6DD21ED2DD122DD9E4FE906FDF
:102B010017E06E601D74802EF8E6FD906F14E0FBF7
:102B1100A3E0FAA3E0F98E82758300ED1204000EA2
:032B210080DC2233
:102DD900CEEFCEE4F56AEE2402FDE433FCE56A6D3C
:102DE9007001EC6010756BDDD56BFD201E03AF6EB5
:0B2DF90022056A80E175D8D57F00221A
:0431ED0075D8D5229A
:0A317E00856DDA75D8C5E4F56C2202
:0A318800856DDA75D8C5E4F56C22F8
:102F0B00C0D075D010E56F700775D8D5C21E800E76
:102F1B00AF6C056C74802FF8E6F5DA75D8C5D0D098
:012F2B002283
:0631D10075D8D5C21E22D4
:102EC600C0D075D010E56C656F700775D8D5C21E79
:102ED600800EAF6C056C74802FF8E6F5DA75D8C5F0
:032EE600D0D02227
:0631D70075D8D5C21E22CE
:0431F10075D8E52286
:10304500E56F14600A04700C75D8D5C21E8008752A
:08305500D8C1800375D8C52223
:0631DD0075D8D5C21E22C8
:102F4C00C0D075D0107480256CF8A6DAE56F140526
:102F5C006C656C700575D8C1800375D8C5D0D0224E
:10309C00C0D075D0107480256CF8A6DA75D8D5C25E
:0430AC001ED0D02240
:0431F50075D8D52292
:0131FC0022B0
:0131FD0022AF
:0131FE0022AE
:0131FF0022AD
:0132000022AB
:0132010022AA
:0132020022A9
:0132030022A8
:0132040022A7
:0132050022A6
:0132060022A5
:0132070022A4
:0132080022A3
:0631E30075D8D5C21E22C2
:03002B00022B2481
:102B2400C0E0C0F0C083C082C0D075D01085D96E1B
:102B3400E5D9131313541F75F003A42431F582E46B
:102B44003428F583E493740193FA740293F912061A
:0C2B54008DD0D0D082D083D0F0D0E03201
:0300000002314882
:0C314800787FE4F6D8FD7581D702213EA7
:1003BA00BB010689828A83E0225002E722BBFE0241
:0903CA00E32289828A83E4932274
:1003D300BB010CE58229F582E5833AF583E02250DF
:1003E30006E92582F8E622BBFE06E92582F8E22229
:0D03F300E58229F582E5833AF583E4932243
:10040000F8BB010DE58229F582E5833AF583E8F032
:10041000225006E92582C8F622BBFE05E92582C8DE
:02042000F222C6
:10042200EFF88DF0A4FFEDC5F0CEA42EFEEC88F01F
:04043200A42EFE22D4
:10043600BC000BBE0029EF8DF084FFADF022E4CCAA
:10044600F875F008EF2FFFEE33FEEC33FCEE9DEC73
:10045600984005FCEE9DFE0FD5F0E9E4CEFD22EDB9
:10046600F8F5F0EE8420D21CFEADF075F008EF2F03
:10047600FFED33FD4007985006D5F0F222C398FDF4
:050486000FD5F0EA2291
:10048B00C2D5EC30E709B2D5E4C39DFDE49CFCEE8C
:10049B0030E715B2D5E4C39FFFE49EFE120436C3CA
:1004AB00E49DFDE49CFC800312043630D507C3E4C5
:0604BB009FFFE49EFE22FB
:1004C100C5F0F8A3E028F0C5F0F8E58215827002C6
:0604D1001583E038F02263
:1004D700A3F8E0C5F025F0F0E582158270021583D8
:0604E700E0C838F0E82235
:1004ED00E88FF0A4CC8BF0A42CFCE98EF0A42CFCAE
:1004FD008AF0EDA42CFCEA8EF0A4CDA8F08BF0A42C
:10050D002DCC3825F0FDE98FF0A42CCD35F0FCEB8A
:10051D008EF0A4FEA9F0EB8FF0A4CFC5F02ECD394F
:0F052D00FEE43CFCEAA42DCE35F0FDE43CFC22BC
:10053C0075F008758200EF2FFFEE33FECD33CDCC76
:10054C0033CCC58233C5829BED9AEC99E5829840F9
:10055C000CF582EE9BFEED9AFDEC99FC0FD5F0D6D6
:10056C00E4CEFBE4CDFAE4CCF9A88222B800C1B900
:10057C000059BA002DEC8BF084CFCECDFCE5F0CB3E
:10058C00F97818EF2FFFEE33FEED33FDEC33FCEB77
:10059C0033FB10D703994004EB99FB0FD8E5E4F932
:1005AC00FA227818EF2FFFEE33FEED33FDEC33FC1F
:1005BC00C933C910D7059BE99A4007EC9BFCE99A13
:1005CC00F90FD8E0E4C9FAE4CCFB2275F010EF2F58
:1005DC00FFEE33FEED33FDCC33CCC833C810D70758
:1005EC009BEC9AE899400AED9BFDEC9AFCE899F893
:0E05FC000FD5F0DAE4CDFBE4CCFAE4C8F92226
:102A1700C2D5E830E70FB2D5E4C39BFBE49AFAE4EA
:102A270099F9E498F8EC30E717B2D5122A4D120558
:102A370078E4C39BFBE49AFAE499F9E498F88003F5
:102A470012057830D50DE4C39FFFE49EFEE49DFD9B
:042A5700E49CFC22DD
:10060A00EB9FF5F0EA9E42F0E99D42F0EC6480C867
:06061A0064809845F02207
:10062000EB9FF5F0EA9E42F0E99D42F0E89C45F030
:0106300022A7
:10063100E8600FECC313FCED13FDEE13FEEF13FFA7
:03064100D8F122CB
:0C064400ECF0A3EDF0A3EEF0A3EFF02229
:10065000A8828583F0D083D08212066712066712C3
:100660000667120667E473E493A3C583C5F0C583E8
:10067000C8C582C8F0A3C583C5F0C583C8C582C8F4
:010680002257
:0C068100A42582F582E5F03583F5832284
:06068D008A838982E473F8
:10005E00E5702434F582E4346FF583E00570229068
:10006E006F31300903906F34E475F0011206B3025C
:10007E0003BA2002E97F2ED2028018EF540F24908B
:10008E00D43440D4FF30060BEF24BFB41A00500313
:10009E002461FFE571600215710574E57470020547
:1000AE007330090E906F31E475F0011206B3EF0252
:1000BE0006930231AA7403D2098003E4C209F570D3
:1000CE00906F311206CAE4F571F573F574E571603F
:1000DE00077F201200A180F5F572C203C202C2048E
:1000EE00C205C207C208C20A12006DFF700D3009A8
:1000FE00057F001200B2AF74AE7322B42561C2D573
:10010E00C20612006DFF24D0B40A00501C75F00A0E
:10011E0020D50DC571A42571F5717002D20580E050
:10012E00C572A42572F57280D724CFB41A00EF5091
:10013E0004C2E5D2060202ACD20380C4D20280BE53
:10014E00D20480BAD2D580B8D20780B27F201200F6
:10015E00A12004077401B5710040F112005EFF1278
:10016E0000A10200DBD20AD208809312005EFB12BD
:10017E00005EFA12005EF94A4B700679787A037BBC
:10018E00FF200433E571602FAF72BF00011F7E00A8
:10019E008E827583001203D360050EEE6F70F1C26E
:1001AE00D5EBC0E0EAC0E0E9C0E0EE1202F0D0E02C
:1001BE00F9D0E0FAD0E0FB1203BAFF60A5EBC0E085
:1001CE00EAC0E0E9C0E01200A1D0E02401F9D0E0DD
:1001DE003400FAD0E0FBE57260DDD572DA80837B05
:1001EE00FF7A0279ECD2048098791080027908C2E5
:1001FE0008C20A8008D2D5790A8004790AC2D5E4E9
:10020E00FAFDFEFF12005EFC7B0820031312005E57
:10021E00FD7B1030020A12005EFE12005EFF7B2094
:10022E00EC3382D592D55013C3E43002069FFFE41F
:10023E009EFEE42003039DFDE49CFCE4CBF8C20388
:10024E00EC700CCFCECDCCE824F8F870F38017C349
:10025E00EF33FFEE33FEED33FDEC33FCEB33FB9966
:10026E004002FB0FD8E9EB300305F8D0E0C448B2EA
:10027E0003C0E00AEC4D4E4F78207B0070C2EAC0FE
:10028E00E01202F2D0F0D0E0200304C4C0E0C4B209
:10029E0003C0F012008AD0F0D5F0EB0200DB12069C
:1002AE00D301795301F758014A4C01464201FB4FE5
:1002BE00020344020349015F4302095501ED460161
:1002CE00ED4501ED47039B50014E2D01522E017558
:1002DE002B01562301732003862A0000016D3F3F38
:1002EE003F00790AA2D5200514300709B91002047F
:1002FE0004B9080104A2D5200802500104200466A6
:02030E00920457
:10031000B571005032C0E07F203005177F30A20455
:1003200072087207500D120347C204C208C2077F49
:1003300030800F300703E9C0E01200A1300703D07E
:10034000E0F9D0E0B571CE3007177F30B9100C124C
:1003500000A17F583006077F788003B90803120098
:10036000A13004057F2D0200A17F20200AF87F2BF9
:100370002008F322920480CF286E756C6C29002D22
:1003800050434958D20312005E3003F8C20378711B
:1003900030D504D2027872F602010C12005E2403FA
:1003A000B405004001E490037F93120092743A1266
:0A03B0000092D2057571040201F7F6
:10307300EFC394094006EFC3940E4004EFB420035A
:05308300D38001C3220F
:102E5600EFC394414006EFC394474018EFC3946113
:102E66004006EFC39467400CEFC394304009EFC3AC
:092E7600943A5003D38001C322F9
:10264100906F10EBF0A3EAF0A3E9F0906F13E0FBB9
:10265100A3E0FAA3E0F91203BAFE906F10E0FBA326
:10266100E0FAA3E0F91203BAFD6E702AED600E9054
:102671006F1674FFF5F01204C145F070037F00225C
:10268100906F11E475F0011204C1906F14E475F0BC
:10269100011204C180B5D3EE6480F8ED64809840E6
:0726A100037F01227FFF22ED
:102FA900E94A4B7001221203BAFF6D700122EF70DA
:0C2FB90004FBFAF92209E970ED0A80EA35
:10168500906F2AEBF0A3EAF0A3E9F0906F2AE0FB54
:10169500A3E0FAA3E0F91203BAFF123073500C90DD
:1016A5006F2BE475F0011204C180E0D201906F2A1E
:1016B500E0FBA3E0FAA3E0F91203BAFF642B600490
:1016C500EFB42D1D906F2AE0FBA3E475F001120421
:1016D500D7A9F0FA1203BA642D6003D38001C3922F
:1016E50001906F2D12065000000000906F2AE0FB5C
:1016F500A3E0FAA3E0F91203BAFF1230E8506A7FBB
:101705000A7E007D007C00906F2DE0F8A3E0F9A330
:10171500E0FAA3E0FB1204EDC8ECC8EDC0E0EEC0B2
:10172500E0EFC0E0906F2AE0FBA3E0FAA3E0F91236
:1017350003BAFF3395E0FEEF24D0FFEE34FFFEE45D
:10174500FCFDD0E0FBD0E0FAD0E0F9EB2FFFEA3E5C
:10175500FEED39FDEC38FC906F2D120644906F2B91
:10176500E475F0011204C18082300110906F2DE004
:10177500FCA3E0FDA3E0FEA3E0FF8011906F2DE048
:0E178500FCA3E0FDA3E0FEA3E0FF1206A522F8
:10069300BB010689828A83F0225002F722BBFE0146
:0206A300F32240
:0E06A500C3E49FFFE49EFEE49DFDE49CFC2266
:1006B300F8E0FBA3A3E0F925F0F0E58215827002D0
:0706C3001583E0FA38F02274
:0906CA00EBF0A3EAF0A3E9F02231
:1006D300D083D082F8E4937012740193700DA3A3B6
:1006E30093F8740193F5828883E4737402936860CA
:0606F300EFA3A3A380DFCA
:1030E800EFC394304009EFC3943A5003D38001C32F
:0130F80022B5
:00000001FF
